:100000008C019D018F019001910192019301940156
:1000100095019601980199019A0183161030850087
:100020000030860064002730810083128C289B01F9
:100030000C089C006D200314980203182A2803144E
:100040000130990203182A28031401309A02031878
:100050002A281B149C031C086D2003149902031802
:100060003728031401309A02031837281B149C0305
:100070001C086D2003149A02031840280314412819
:100080001B0C00349B010C089C006D20031098078A
:10009000031C5528031001309907031C5528031031
:1000A00001309A07031C55281B149C031C086D2063
:1000B00003109907031C6228031001309A07031CE0
:1000C00062281B149C031C086D2003149A07031C50
:1000D0006B2803146C281B0C003482070034003496
:1000E0000A3400340034643400340334E834003417
:1000F0002734103401348634A0340F344234403471
:1001000082073F3406345B344F3466346D347D34BB
:1001100007347F34673480348316003086008312BE
:1001200011308C0009308D008E0106309D001720A3
:100130000318A1288E0A8D03031D972803308C0213
:10014000A428422003308C0209308D0010301D0796
:100150009B009B031B0884000E088E0180009D03FA
:1001600001300C07031D972818088F0097018101A3
:10017000000000009D013C308C008B011030850098
:1001800083161830850083120F301D078400000885
:1001900080209B00053003151D02031DD0289B17EE
:1001A0001B0886001D08000085000B1DDA28970A31
:1001B0000B11DD2800000000000007309B009B0BA6
:1001C000DF2800009D0A073003111D02031DC4280B
:1001D000000003309B009B0BEB2800009D018C0B63
:1001E000C428000031309B009B0BF4280000000065
:1001F0000B1DFD28970A0B110029000000000000CC
:1002000003018600103085008316103085008312AC
:100210000B19970A0B110108990017089A009B0106
:100220009B0A851585110B11010803111902031989
:0E02300010299B0A9B099B0A1B0A98008C2828
:00000001FF
